S018000064656D6F70726F675F7333326B3131382E7372656373
S1132000005800203D250000992500009925000076
S113201000000000000000000000000000000000BC
S113202000000000000000000000000099250000EE
S1132030000000000000000099250000D92C0000D9
S11320409925000099250000992500009925000094
S11320509925000099250000992500009925000084
S11320609925000099250000992500009925000074
S11320709925000099250000992500009925000064
S11320809925000099250000992500009925000054
S11320909925000099250000992500009925000044
S11320A09925000099250000992500009925000034
S11320B09925000099250000992500009925000024
S10720C0EE11AA551A
S1132400FFFFFFFFFFFFFFFFFFFFFFFFFE7FFFFF59
S1132410054B0648033310B51B1A062B03D9044B8E
S1132420002B00D0984710BD28010020280100206F
S1132430000000000648074910B5091A8910CB0F9F
S11324405918491003D0044B002B00D0984710BDF5
S113245028010020280100200000000010B5074CCE
S11324602378002B09D1FFF7D3FF054B002B02D0B3
S1132470044800E000BF0123237010BDC0300020D9
S113248000000000382F0000094B10B5002B03D0CA
S11324900849094800E000BF08480368002B02D13E
S11324A0FFF7C8FF10BD064B002BF9D09847F7E79C
S11324B000000000C4300020382F00002401002058
S11324C000000000164B002B00D1144B9D46402207
S11324D092029A1A924600218B460F461348144AD8
S11324E0121A00F0F9FC0F4B002B00D098470E4B4A
S11324F0002B00D098470020002104000D000D4857
S1132500002802D00C4800E000BF00F0C1FC20000D
S1132510290000F05DFB00F0A5FCC04600000800A7
S1132520005800200000000000000000C03000201F
S113253034310020000000000000000072B6104991
S11325400F4A0F4B0E4C0E4D0D4E0D4FB846B9466B
S1132550BA46BB46BC460B490B4A521A013A05DD42
S11325600020042308601944043AFBDA074885462E
S1132570074880470748804762B6FFF7A3FFFEE796
S11325800000000000000020005800200058002037
S1132590E92C0000892D0000FEE7C0460022430814
S11325A08B4274D303098B425FD3030A8B4244D317
S11325B0030B8B4228D3030C8B420DD3FF22090259
S11325C012BA030C8B4202D31212090265D0030B18
S11325D08B4219D300E0090AC30B8B4201D3CB030E
S11325E0C01A5241830B8B4201D38B03C01A524150
S11325F0430B8B4201D34B03C01A5241030B8B4252
S113260001D30B03C01A5241C30A8B4201D3CB023C
S1132610C01A5241830A8B4201D38B02C01A524121
S1132620430A8B4201D34B02C01A5241030A8B4224
S113263001D30B02C01A5241CDD2C3098B4201D33C
S1132640CB01C01A524183098B4201D38B01C01ABA
S1132650524143098B4201D34B01C01A5241030931
S11326608B4201D30B01C01A5241C3088B4201D3E0
S1132670CB00C01A524183088B4201D38B00C01A8D
S1132680524143088B4201D34B00C01A5241411AB4
S113269000D20146524110467047FFE701B50020C1
S11326A000F006F802BDC0460029F7D076E770476F
S11326B07047C04670B50C4B1B68002B00DB70BD27
S11326C0094A13685B005B08136000F0FFFAFA30F4
S11326D00400054E80256D0333682B42EFD000F0D3
S11326E0F5FA8442F8D2EAE70040024070B50D4B97
S11326F019688022D2050A431A601968802252059B
S11327000A431A6000F0E2FAFA300400054E80250C
S11327106D0433682B4203D100F0D8FA8442F8D216
S113272070BDC04600400240F0B585B0002302AA47
S1132730137001335370013393700233D370043335
S1132740137108335371103393712033D371AA4A30
S11327506933FF33D158A9480140D150D05884215E
S1132760C9050143D1505C33A54AD3585B055B0FBF
S113277005D18021490081239B00D150012382226D
S113278092009F498A58D20776D49E4802AAD15C07
S1132790FFF704FFE1210902FFF700FFC31D1B043B
S11327A0DB0CE022D2041A43974B1A61974A5A6110
S11327B000229A611A625A62F02292029A629A6A1A
S11327C088210A439A620122DA62C02212039A61C2
S11327D08949902288588023DB0503438B50FFF7F7
S11327E069FFFFF783FF8A4B1B68002B13DB884AC2
S11327F0116880231B060B43136000F067FAFA305C
S11328000400834E80256D0333682B4203D100F00E
S11328105DFA8442F8D27E4A53687E490B40536085
S1132820FFF748FFFFF762FF002302AA137001338A
S11328305370013393700233D3700433137108332C
S11328405371103393712033D371C4336C4AD3580A
S11328505B055B0F06D1802149000533FF33D1505E
S1132860043BFF3B02AAD15C6B48FFF797FE019043
S11328706A4F0026002505E0694887E701360437DA
S1132880122E1BD03A785401A41AA400A418A40050
S113289021000198FFF708FF0029EFD121000198DA
S11328A0FFF77CFE85B26B1E9BB2FF2BE6D8B60009
S11328B05A4B9E197778B078F17802E00021002015
S11328C00027534A5468574B1C40546054686B1E8D
S11328D01B062343536056687D1E07232B40334356
S11328E053605468431EDB04E025AD032B402343AF
S11328F0536054684B1E1B04E021C9020B40234360
S113290053605268031C042800D90423DBB2013B42
S11329109B05C02109040B4013433D4A536053688F
S113292080210B4353600023100000211A00203241
S1132930920011500133802BF8D100233448002138
S1132940882292009A18920011500133202BF7D15B
S11329502F4B1A687F218A4360390A431A60196829
S1132960802292020A431A601968802252020A43A2
S11329701A601A682C490A401A602C492C4A99504A
S11329808021C9048822520099502A49043299505E
S113299000229A62013A1A63274A1A621A6827497E
S11329A00A401A605A6826490A405A601A6813494C
S11329B00A401A601A6823490A401A6000F086F92E
S11329C0FA300400124E80256D0433682B4203D084
S11329D000F07CF98442F8D200F078F9FA3004006F
S11329E00B4E80252D0533682B4203D000F06EF981
S11329F08442F8D205B0F0BD00500640FFFFFFBF8F
S1132A000040064080841E0000A0064000C01FC095
S1132A1000400240FFDFFFFF409C0000EC2E00005E
S1132A2000127A0078FF0000FFFFFFDFFFFFFF5F67
S1132A30A408000000009C1906003B00FFFF7FFF74
S1132A40F7EFFFFFFFFFFFEF30B583B03A4B1B7882
S1132A50002B3AD1394B5B699B0207D5374BDB69B5
S1132A60DBB2374A1370013B3F2B23D9354B1B6B29
S1132A709B051DD588235B00324AD1580903090FF1
S1132A8052D00023032430481A006240D2B2125CB0
S1132A906D465A550133DAB29142F5D8294B80225A
S1132AA092001A639A68294B1A602B78FF2B2BD05B
S1132AB003B030BD00F00AF9254B186001221E4B0B
S1132AC01A700022234B1A70D0E71C4B5B699B02DF
S1132AD01FD520490B78194AD469194AD018447073
S1132AE00133DBB20B7012789A42BFD10022124B31
S1132AF01A70134B5B78FF2BB8D1114B9B78002BCA
S1132B00B4D100F031F9B1E70229D1D100F02CF9A8
S1132B10CEE700F0DBF80E4B1B6864339842A5D96E
S1132B200022054B1A70A1E7064B802292001A631B
S1132B309A68064B1A60BBE72131002000A00640CA
S1132B40E03000200040024018410240DC30002008
S1132B50243100202231002080235B00044A1362C8
S1132B60044A51691943516191680B43936070475A
S1132B7000D0044000F10F4010B500F0A7F8114B4D
S1132B801B68C31AF422FF3293420FD90E4B1B78F1
S1132B90002B0CD1F33AFF3A0B4B1A700B4A5168D5
S1132BA080235B000B435360064B186010BD00226A
S1132BB0054B1A70054A916880235B000B439360B0
S1132BC0F2E7C0462C3100202831002000F10F40EC
S1132BD010B52D4B0221FF31822252009950CD397C
S1132BE0043299501900083A80231B04885818426B
S1132BF0FCD1012180235B00234AD15011001A002B
S1132C0080235B0488581842FCD01F4B0222FF32F9
S1132C10C12189005A500139FF395A501B4A5A615F
S1132C2019000F220B691B0E1340032BFAD100F07D
S1132C306DF8174B9420400019588022D205114397
S1132C4019509A214900585802435A50114B196897
S1132C50802292001143196059680A435A600E4B4E
S1132C601969A022D2001143196159690A435A61B2
S1132C7000F014F8FFF770FF62B6FFF755FDFFF799
S1132C807BFFFFF7E1FEFAE7004006400100000386
S1132C900050064000A0044000D0044010B5084B8A
S1132CA01868FA218900FFF779FC0138054B586050
S1132CB000229A6007211960034B1A6010BDC046B8
S1132CC0C000002010E000E030310020014B186803
S1132CD07047C04630310020024A13680133136044
S1132CE07047C04630310020044B054A5A605A6888
S1132CF0044A1A60044A9A607047C046002005409E
S1132D0020C528D920210000FFFF000010B5124B78
S1132D1019691B691B011B0F022B0CD0032B12D04A
S1132D20012B07D10D480903090F0131FFF736FCC8
S1132D300B4B186010BD82239B00074AD358DB0756
S1132D40F8D50648EFE7C2239B00034AD3589B07F4
S1132D50F0D10448E7E7C0460040064000127A007C
S1132D60C0000020006CDC020448054943581B04E1
S1132D701B0C044A134343507047C04600E000E074
S1132D800C0D00000400FA0530B5274A274B9A427F
S1132D9009D02649891A0023254C1000C25CE2544C
S1132DA001338B42FAD1234A234B9A4209D0224958
S1132DB0891A0023214C1000C25CE2540133994269
S1132DC0FAD11F4A1F4B9A4206D0130000211D4A14
S1132DD0197001339342FBD11B4A1C4B9A4209D010
S1132DE01A49891A00231A4C1000C25CE2540133B8
S1132DF09942FAD1174A184B9A4210D017498908B8
S1132E0009D000230022134C1348C558E550013261
S1132E1004338A42F9D1124B0E4A1A6030BD104B6A
S1132E200D4A1A60FAE7C046602F0000C82F000060
S1132E30C0000020C82F0000C82F00002801002077
S1132E40C030002034310020C82F0000C82F0000FB
S1132E50C03000200000002000200000C00000005E
S1132E6008ED00E0084B10B50400002B02D000214F
S1132E7000E000BF054B1868836A002B00D0984718
S1132E80200000F031F8C04600000000342F00009C
S1132E9070B500260C4D0D4C641BA410A64209D13C
S1132EA0002600F049F80A4D0A4C641BA410A642FF
S1132EB005D170BDB300EB5898470136EEE7B30077
S1132EC0EB5898470136F2E7582F0000582F0000BE
S1132ED0582F00005C2F000003008218934200D199
S1132EE0704719700133F9E7FEE700000803020296
S1132EF0090303020A0303030B0403030C0404037E
S1132F000D0504030E0504040F060404100605044D
S1132F10110705041207050513080505140806051D
S1132F2015080705160807061708080618080807ED
S1132F3019080808C4000020F8B5C046F8BC08BC4D
S1132F409E467047F8B5C046F8BC08BC9E4670471C
S10B2F5074F5FF7F010000008D
S1072F5889240000C4
S1072F5C5D240000EC
S1132F60006CDC0200000000000000000000000013
S1132F70000000000000000000000000000000004D
S1132F80000000000000000000000000000000003D
S1132F90000000000000000000000000000000002D
S1132FA0000000000000000000000000000000001D
S1132FB0000000000000000000000000000000000D
S10B2FC0000000000000000005
S903253D9A
